:100000000C9462000C94B91A0C94E61A0C948A00B1
:100010000C948A000C948A000C948A000C948A0038
:100020000C948A000C948A000C948A000C948A0028
:100030000C948A000C94800B0C948A000C948A0017
:100040000C94131B0C948A000C948F1E0C94D21EDB
:100050000C948A000C948A000C948A000C948A00F8
:100060000C94E1080C948A000000000700020100D3
:100070000003040600000000000000000102040864
:100080001020408001020408102001020408102002
:10009000040404040404040402020202020203032E
:1000A00003030303000000002300260029000000D2
:1000B0000000250028002B0000000000240027007D
:1000C0002A00C01F11241FBECFEFD8E0DEBFCDBF76
:1000D00012E0A0E0B1E0E4EFF1E402C005900D927F
:1000E000A23DB107D9F714E0A2EDB2E001C01D9224
:1000F000AC3BB107E1F710E0C4ECD0E004C02297BC
:10010000FE010E94D520C23CD107C9F70E94FC1F06
:100110000C94F8200C9400008091BE03813019F4F7
:1001200082E08093BE038091BE03833019F484E0A3
:100130008093BE030895A8950895CF93DF93FC01A3
:10014000962F9270862F817060FF20C0992331F026
:100150008091500380831092D20216C0A091D202E7
:10016000C091E903C770D0E0C656DD4F8881A8175B
:1001700010F080E03CC081E08A0F8093D202B0E0B2
:10018000A050BD4F8C91808381E031C09923C1F094
:1001900090819093D3021092D202292F207E203694
:1001A00051F490915003923020F390819F7190937D
:1001B000920393E01AC09E3F39F71092500317C084
:1001C0009091D3029F3F01F79091D202993288F625
:1001D00021E0290F2093D2023081E92FF0E0EF5384
:1001E000FC4F3083293281F691E090935003DF91E8
:1001F000CF910895DC01ED91FC910190F081E02D0B
:1002000009950895DC01ED91FC910190F081E02DBC
:10021000099508952091BF033091C003382748E025
:10022000C901880F991F37FF06C09C0151E225279D
:1002300050E1352701C09C01415091F73093C00334
:100240002093BF0308958436910520F4BC0180E01B
:1002500090E017C09C018E3B910528F42A55310986
:10026000AAE0B0E00CC0823D910528F4245B31097E
:10027000A4E6B0E004C02D5C3109A8E5B2E00E941C
:100280000920A4E6B0E09B01AC010E94182008956B
:1002900090E08C599F4F0E942301089585E0809340
:1002A000EA0380E28093EB0382E28093EC0381E235
:1002B0008093ED0383E28093EE038BE28093F0035F
:1002C00084E28093F10385E28093F203089560E075
:1002D0008CE00E94211C61E08BE00E94211C61E007
:1002E0008DE00E94211C60E082E00E94211C61E000
:1002F00084E00E94211C089542E050E06CE870E028
:1003000080E00E94991A0895E3E0F0E089E080938C
:100310005700E491E67081E0E63009F080E008954E
:10032000CF93DF93C82F0E948401882381F0DFB729
:1003300081E08093BD03F8940E949B0088E1809344
:100340006000C0936000C1110E949B00DFBFDF917D
:10035000CF910895FC0140A5842F877090E095957A
:1003600087950196242F217030E0820F931F880F0C
:10037000880F08958F929F92AF92BF92CF92DF9293
:10038000EF92FF92CF93FC01C0A5EC2FE770F0E055
:10039000E656FD4FA081B0E0C7FF03C024E130E086
:1003A00002C02FE030E0FC0197A183E1989FF001AB
:1003B0001124E25AFE4F80809180A280B380A20F68
:1003C000B31F20E43FE14DE750E00E942320A50148
:1003D00094010E945B208C2F887149F469017A0195
:1003E000E0EDCE0EE7E0DE1EE11CF11C1BC0C7FFF6
:1003F00005C060E47AE88CE29EE004C060E07EEE36
:100400008AEB9BE069017A01F8EBCF0EFBE0DF1E7F
:10041000E11CF11CA50194010E945B20C20ED31EB9
:10042000E41EF51EC701B60169517C4F8F4F9F4FE7
:1004300028EE33E040E050E00E945B20A8EEB3E0FD
:100440000E941820CF91FF90EF90DF90CF90BF9047
:10045000AF909F908F900895DB01FA01582F569529
:1004600090E02481237030E0322F22274081240F36
:10047000311D11963C932E9344814C70218130E0C4
:1004800060E4469F200D311D112413963C932E935A
:10049000129744814073228130E060E1469F200D35
:1004A000311D112415963C932E9314974481407C62
:1004B000238130E064E0469F200D311D1124179602
:1004C0003C932E931697359618969F5F591748F6CA
:1004D00080FF47C0408142954695469543702DE484
:1004E00031E0429FC001439F900D11240C9611965C
:1004F0009C938E93808190E074E0969587957A9591
:10050000E1F783709927829FA001839F500D929FEE
:10051000500D1124445F5F4F13965C934E931297D6
:10052000808190E096958795969587958370992719
:10053000829FA001839F500D929F500D1124445F14
:100540005F4F15965C934E93149740814370429F82
:10055000C001439F900D11240C9617969C938E9387
:1005600016970895803223E0920708F1883E23E031
:10057000920740F48F519340E4E096958795EA9571
:10058000E1F70895803D27E0920718F48C5D9340D1
:100590000895883928E0920768F4885C974074E0F1
:1005A000969587957A95E1F78D509C4F089580E058
:1005B00090E008958FEF93E008958C30910540F41A
:1005C000A4E0880F991FAA95E1F7885D9C4F0895D4
:1005D000843F23E0920718F484529C4F08958115BC
:1005E00024E0920740F48657934FF4E0880F991F58
:1005F000FA95E1F7089580E998E008959C01369511
:10060000279525753575821B930B9C0123733373D6
:10061000969587959695879583739373820F931F0D
:100620009C0154E0369527955A95E1F7280F391F1C
:100630002F703F7041E051E0249FC001259F900D35
:10064000349F900D1124892F08952D98882319F037
:1006500000002B9A02C000002B9800002D9A000089
:1006600008952D9A000083B12D9800008295817025
:100670000895CF93DF93D82F5C9A2D985C98C8E0AB
:100680008D2F80780E942503DD0FC150C9F72D986A
:10069000DF91CF9108958F770E9439030895CF930A
:1006A000DF93D82FC8E08D2F80780E942503DD0FBF
:1006B000C150C9F72D98DF91CF910895CF93DF9363
:1006C0002D98C8E080E0D82FDD0F0E9431038D0FF8
:1006D000C150C9F7DF91CF9108950E944B030E944A
:1006E0005E035C9A0895A1E0B0E0E9E7F3E00C94C2
:1006F000AC20806869830E9439036981862F0E943B
:100700004F035C9A2196E2E00C94C820CF93C091ED
:10071000CA03C827E82FF0E0EF53FC4F678589E74D
:100720000E9473036C2F8DE30E9473036C2F82E48D
:100730000E947303CF91089586E20E946D0308958D
:10074000CF938BE20E946D03C82F8CE20E946D0351
:10075000282F30E066E0369527956A95E1F744E06A
:10076000C49FC0011124822B932BCF910895CF9366
:10077000DF93EC016C818CE10E9473036D818DE14C
:100780000E9473036E818EE10E9473036F8180E289
:100790000E947303688581E20E947303698582E287
:1007A0000E9473036A8583E20E9473036B8584E26F
:1007B0000E9473036C8585E20E9473036D858AE253
:1007C0000E9473036E858EE60E9473036F858FE629
:1007D0000E947303688980E70E947303698981E737
:1007E0000E9473036A8982E70E947303DF91CF91AD
:1007F0000895CF92DF92EF92FF92CF93DF936B0138
:100800007C01C11488E3D8068CE9E8068CE1F8067F
:1008100028F5C701B60120E836E948E950E00E9412
:100820005B20E901689760E879E687E69FEF0E9420
:100830002B206C0D7D1D8E1D9F1DF2E0660F771F16
:10084000881F991FFA95D1F721E732E040E050E088
:100850000E945B20F22EE32E80E421C0C701B60186
:1008600020E03DE241E351E00E945B20E90168970E
:1008700060E073ED8EEC9EEF0E942B206C0D7D1DD1
:100880008E1D9F1D660F771F881F991F21E732E07D
:1008900040E050E00E945B20F22EE32E80E66C2FB9
:1008A0006F71680F85E70E9473036E2D86E70E94C3
:1008B00073036F2D87E70E947303DF91CF91FF9041
:1008C000EF90DF90CF9008958F929F92AF92BF925A
:1008D000CF92DF92EF92FF92CF93DF93D82F83E0F6
:1008E0000E946D038093BC0384E00E946D0380939B
:1008F000BB0360E086E00E94730361E087E00E9432
:1009000073036FE789E00E94730365E08AE00E9449
:10091000730362E18BE00E94730365E18CE00E9447
:1009200073036DEF8DE00E94730360E08EE00E9420
:100930007303DD2319F08BE491E008C02091E803F4
:1009400033E1239FC0011124825A9E4F0E94B703B6
:100950006CE880E30E9473036FE082E30E947303FC
:1009600062E483E30E9473038091E90387FF02C07E
:1009700064E101C06AE084E30E9473036AE285E3F4
:100980000E9473036DE286E30E94730364ED87E3C4
:100990000E94730360E088E30E94730360E089E3D0
:1009A0000E947303D11109C0C090CA03D090CB0339
:1009B000E090CC03F090CD0307C0C5E9CC2EC1EC8C
:1009C000DC2EED2CCEEDFC2ECAE38F2C9924AA242C
:1009D000BB24682D8C2F0E947303682D85E08C0F3B
:1009E0000E947303FE2CED2CDC2CCC24CF5FCE3385
:1009F00061F76FEF83E40E9473036FEF84E40E945A
:100A000073036FEF85E40E9473036FEF86E40E9427
:100A10007303DD2311F066E002C06091CE038DE622
:100A20000E94730360E089E70E9473036091CF0323
:100A30008AE70E94730360E083E70E94730360E02B
:100A400084E70E947303D11109C06091C6037091BD
:100A5000C7038091C8039091C90304C060E071EAA4
:100A60008CEB93E30E94F903DF91CF91FF90EF901D
:100A7000DF90CF90BF90AF909F908F90089561E0EE
:100A800087E00E94730364E28EE70E94730363E0D1
:100A900088E00E94730360E088E00E94730365E0D1
:100AA00087E00E94730362E085E00E94730383E0A5
:100AB0000E946D038093BC0384E00E946D038093C9
:100AC000BB03089583E00E946D038093BC0384E020
:100AD0000E946D038093BB0361E087E00E94730373
:100AE0006AE070E080E090E00E948C1B0E943F056D
:100AF00000000895CF92DF92FF920F931F93CF9340
:100B0000DF931F92CDB7DEB7082F162F8EE39983A0
:100B10000E947303F02EC02E9981D92E8C2D8F192F
:100B2000811738F4F60161916F018FE70E9473031A
:100B3000F5CF64E085E00E94730383E00E946D03BB
:100B40008093BC0384E00E946D038093BB030E94EA
:100B5000691B6093B7037093B8038093B9039093B4
:100B6000BA0369E087E00E94730381E08093BE03CB
:100B70000F90DF91CF911F910F91FF90DF90CF9059
:100B800008950F931F930E947A058091BE038130D0
:100B900099F40E94691B0091B7031091B80320914A
:100BA000B9033091BA03601B710B820B930B603A4F
:100BB00076488140910548F38091BE03813031F43D
:100BC0006EEB71E082E194E00E942B1D1F910F916A
:100BD00008950F931F938091BE03823021F41092E9
:100BE000BE0381E020C08091BE038130D9F40E9411
:100BF000691B0091B7031091B8032091B90330919C
:100C0000BA03601B710B820B930B613A76488140EB
:100C1000910540F061E087E00E9473031092BE03EB
:100C200082E001C080E01F910F910895EF92FF9242
:100C30000F931F93CF93DF938B019C01442737FDC4
:100C40004095542F60E271EA87E090E00E947D2099
:100C5000E9011C161D0614F0C1E0D0E0D80120E225
:100C600031EA47E050E00E9423209E01442737FDEF
:100C70004095542F0E947D20790100E010E00E1570
:100C80001F055CF42B9ACE010E94B21B2B98CE015B
:100C90000E94B21B0F5F1F4FF2CFCDB7DEB7E6E069
:100CA0000C94C420CF93DF935D9A6091FA03709106
:100CB000FB038091FC039091FD030E94F90360E027
:100CC00089E70E94730361E070E080E090E00E9499
:100CD0008C1B0E949C03C82F61E070E080E090E0D4
:100CE0000E948C1B0E949C03D0E0C80FD11D61E0C4
:100CF00070E080E090E00E948C1B0E949C03C80F73
:100D0000D11D61E070E080E090E00E948C1B0E94A9
:100D10009C035D989E01280F311DC901969587950A
:100D200096958795DF91CF910895CF93C82F5D9ABF
:100D300083E00E946D038093BC0384E00E946D03F6
:100D40008093BB0360E086E00E94730361E087E06C
:100D50000E9473036FE789E00E94730365E08AE0F5
:100D60000E94730362E18BE00E94730365E18CE0F3
:100D70000E9473036DEF8DE00E94730360E08EE0CC
:100D80000E9473036CE280E70E94730360E080E3DB
:100D90000E94730360E089E70E94730365E08AE7BD
:100DA0000E94730362E181E70E94730362E082E7BD
:100DB0000E94730360E083E70E94730360E084E7AE
:100DC0000E9473036091FA037091FB038091FC030E
:100DD0009091FD030E94F90367E08DE60E94730382
:100DE0006AE070E080E090E00E948C1B69E087E0A0
:100DF0000E9473036AE070E080E090E00E948C1B28
:100E0000CC2369F0C5E1C15009F459C061E070E03C
:100E100088EB91E00E9416060E949B00F4CF61E0EF
:100E200070E088E891E00E9416060E949B0065E051
:100E30008DE60E9473036AE070E080E090E00E941B
:100E40008C1B61E070E088EB91E00E9416060E9426
:100E50009B0064E08DE60E9473036AE070E080E02E
:100E600090E00E948C1B61E070E08DE591E00E94B3
:100E700016060E949B0062E08DE60E9473036AE002
:100E800070E080E090E00E948C1B61E070E08FEAEF
:100E900090E00E9416060E949B0060E08DE60E9492
:100EA00073036AE070E080E090E00E948C1B62E0D7
:100EB00070E085E091E00E9416060E949B0061E0D0
:100EC00087E00E9473035D98CF910895CF93DF93DD
:100ED000EC014AE050E06D2F70E082E194E00E9466
:100EE000F01D6EE282E194E00E940F1DBE0184E0DD
:100EF000769567958A95E1F76F7077274AE050E01D
:100F000082E194E00E94F01DDF91CF910895D82FE7
:100F1000C0E0CD1780F45E9A64E670E080E090E077
:100F20000E948C1B5E9864E670E080E090E00E9476
:100F30008C1BCF5FEECF6CE271E080E090E00E940E
:100F40008C1BE6CF0F931F93CF93DF93EC01062FFB
:100F500015E0115051F0CE010E94E220081741F037
:100F6000602FCE010E94EA20F4CF82E00E94870722
:100F7000DF91CF911F910F910895A0E0B0E0E3ECD5
:100F8000F7E00C949E20482E562EC0E0D0E0612C55
:100F9000712CE12CF12C00E010E0442079F081E08C
:100FA0004816A1F092E0491219C028E4622E712C73
:100FB00030E2E32EF12C03E513E010C0612C712C1C
:100FC0006BE1E62EF12C0AEE13E008C04DE1642E31
:100FD000712C59E2E52EF12C01EC13E043018C0E4B
:100FE0009D1E1092C0031092BF033401A62CA818B6
:100FF000B12CC30101966C01AE14BF04A8F4A00E7D
:10100000B11E511006C0C3010E94E220F501808389
:1010100005C0F5016081C3010E94A207F50180812E
:101020000E940A013601E2CFC301511018C0C3016A
:101030000E94E220B82EC6010E94E2202B2D30E053
:10104000322F2227282B8091BF039091C003821753
:10105000930779F4C0E0D0E0552453949ECF360135
:101060006091C0030E94A2076091BF03C6010E9465
:10107000A207D395C13093E0D90708F48ECF852D10
:10108000CDB7DEB7E0E10C94BA2060E081E00E94C9
:10109000BD07882331F081E09091C103983309F0B6
:1010A00080E0089561E081E00E94BD07089561E05D
:1010B00082E00E94BD07089560E082E00E94BD07C3
:1010C000811108C0E3E5F3E01192119283E0E33768
:1010D000F807D1F70895A1E0B0E0E1E7F8E00C945B
:1010E000AC2089830E944E0192E09093F8039FEF19
:1010F0009093F9039AE090930204109203041092E3
:1011000004041092FA031092FB031092FC03109255
:10111000FD032EE12093FE039093FF0328EB3BE0B9
:1011200030930104209300048981882371F061E0E9
:1011300080E00E94BD07E3E5F3E01192119283E0A5
:10114000E337F807D1F70E9457082196E2E00C94A4
:10115000C82060E080E00E94BD07811103C081E0EB
:101160000E946B080895CF93C1E0811101C0C0E0D7
:101170006C2F82E10E945A1C6C2F83E10E945A1C42
:101180001092B1031092B0038091B9008C6F8093DC
:10119000B90080E28093B80085E48093BC00CF91D1
:1011A000089585ED8093BC008091BC0084FDFCCF48
:1011B0000895ECEBF0E0108285E480831092B00398
:1011C00008951F920F920FB60F9211242F933F9301
:1011D0004F935F936F937F938F939F93AF93BF933F
:1011E000EF93FF93CF93DF931F92CDB7DEB780913C
:1011F000B900887F803609F4C7C0A8F5883209F4A1
:1012000064C098F4803109F45DC038F4882309F48F
:10121000F3C0883009F456C0F1C0883109F455C0D4
:10122000803209F0EBC082E0A7C0803409F477C0B7
:1012300078F4803309F45FC0883309F0DFC084E0BC
:101240008093AF038091B0038B7F8093B003D0C0B5
:10125000803509F452C0883509F467C0883409F034
:10126000CDC085E089C0883909F4C0C0A8F48837AA
:1012700009F48AC038F4883609F486C0803709F446
:1012800083C0BCC0883809F4B1C0803909F47FC07C
:10129000803809F0B3C07BC0803B09F493C038F4B8
:1012A000803A09F48CC0883A09F48CC0A7C0803C0D
:1012B00009F49EC0883C09F49BC0883B09F09EC09D
:1012C00080E081C08091B40313C08091B1039FEF8F
:1012D000980F9093B1038823D1F1E091B203F0917C
:1012E000B303CF0101969093B3038093B20380813F
:1012F0008093BB007DC083E03FC0E091B203F091DA
:10130000B303CF0101969093B3038093B20380910E
:10131000BB0080838091B10381508093B1038091A1
:10132000B103823008F064C061C0E091B203F09173
:10133000B303CF0101969093B3038093B2038091DE
:10134000BB0080838091B10381508093B103809171
:10135000B0038B7F8093B0038091B00380FF4CC0BB
:101360008091B0038E7F8093B0038091B003826040
:101370008093B00384EA3DC08093AF038091B003B3
:101380008B7F8093B00338C01092B10331C0E091DD
:10139000B503F091B603309749F18091BB00898382
:1013A0008091B10391E0980F9093B103811102C035
:1013B00062E001C060E0CE010196099515C00E946F
:1013C000D10816C081E0E091B503F091B6033097E3
:1013D00069F0882311F063E001C061E0CE0101965D
:1013E000099599819093BB00811102C085E801C0E5
:1013F00085EC8093BC0002C00E94D1080F90DF9161
:10140000CF91FF91EF91BF91AF919F918F917F917C
:101410006F915F914F913F912F910F900FBE0F9061
:101420001F9018958F929F92AF92BF92CF92DF92AA
:10143000EF92FF92CF93DF93EC010E94691B6B0147
:101440007C014E01A12CB12C8091B00382FF11C010
:101450002097D1F30E94691B6C197D098E099F09A1
:1014600086169706A806B90678F70E94D90881E083
:1014700004C08091AF031092AF03DF91CF91FF9032
:10148000EF90DF90CF90BF90AF909F908F90089596
:10149000A2E0B0E0EEE4FAE00C94A820182F7B0163
:1014A000022F047022FD05C080910B0190910C0168
:1014B00002C080E090E02A8349830E94120A2A81B8
:1014C0004981811136C01092AF034093B103F0926D
:1014D000B303E092B203110F1093B4039091B003E1
:1014E00021FF02C085E001C084E0892B8093B00316
:1014F0008091B00381FF0BC08091B0038D7F8093FA
:10150000B0038091B4038093BB0085EC01C085EEED
:101510008093BC00822F817020FF0BC0011105C099
:1015200080910B0190910C0102C080E090E00E943C
:10153000120A2296E6E00C94C420A2E0B0E0E3EAAE
:10154000FAE00C94A820182F7B01022F047022FDD2
:1015500005C080910B0190910C0102C080E090E0E9
:101560002A8349830E94120A2A814981811138C045
:101570001092AF034093B103F092B303E092B20331
:10158000812F880F81608093B4039091B00321FF75
:1015900002C085E001C084E0892B8093B003809174
:1015A000B00381FF0BC08091B0038D7F8093B003A7
:1015B0008091B4038093BB0085EC01C085EE8093DD
:1015C000BC00822F817020FF0BC0011105C08091EB
:1015D0000B0190910C0102C080E090E00E94120A81
:1015E0002296E6E00C94C420A0E0B0E0EAEFFAE036
:1015F0000C94A6200E94691B0091AB031091AC03D0
:101600002091AD033091AE036B017C01C01AD10A69
:10161000E20AF30A9701860141E1C41647E2D406C3
:10162000E104F10408F442C02091AA0331E0320F32
:101630003093AA0320FF02C017E001C010E06093BE
:10164000AB037093AC038093AD039093AE0363E060
:1016500070E082E194E00E94020161E070E082E1CA
:1016600094E00E94020107E0010F812F90E0EC015D
:10167000CC0FDD1FC35FDE4F68817981672F77272D
:1016800063707727880F991F880F991F682B792B14
:1016900082E194E00E94FA0068817981772782E1F3
:1016A00094E00E94FA001F5F1013DFCFCDB7DEB7C2
:1016B000E8E00C94C22025B190E0FC01EE0FFF1F82
:1016C000E80FF91FE65EFC4F8081282B25B988B111
:1016D0009181892B88B98BB19281892B8BB908951F
:1016E00085B190911703892385B988B1909118032A
:1016F000892388B98BB19091190389238BB90895F7
:101700001F920F920FB60F9211242F933F934F9376
:101710005F936F937F938F939F93AF93BF93CF9379
:10172000EF93FF93C091760380910601C81708F0EC
:101730003EC080911503909116039093870080938B
:101740008600EC2FF0E0EE0FFF1FE35FFE4F80817D
:1017500091810E94DD02880F991F90931603809358
:101760001503809115039091160320910701309184
:101770000801281B390B3093080120930701809141
:10178000000490910104880F991F2817390720F44D
:10179000909308018093070180917403811142C0E6
:1017A0008091F80380FF41C0C830E0F53EC08091D1
:1017B0001503909116039093870080938600809183
:1017C000070190910801909316038093150380916F
:1017D0007403882319F08FEF9FEF06C080911503E3
:1017E00090911603885592409093890080938800C9
:1017F00080E49CE990930801809307018091840024
:10180000909185008097D0F30E94700B80917503B2
:10181000811105C08091060181500E945B0B1092DE
:10182000760327C08FEF9FEF06C08091150390913C
:101830001603885592409093890080938800809188
:101840008400909185008097D0F30E94700B809166
:101850007503811104C080917603811106C08091C7
:1018600076038F5F8093760304C081500E945B0BE8
:10187000F6CFFF91EF91CF91BF91AF919F918F9153
:101880007F916F915F914F913F912F910F900FBE7C
:101890000F901F90189524E0829FC00111248C3076
:1018A000910538F0853F23E0920728F084EF93E01C
:1018B00008958CE090E00895CF93DF93C091F903F1
:1018C000C03390F48C2F807339F0803141F48091D3
:1018D00077038295807F05C080917C0302C0809150
:1018E0007D03CF70D0E015C0CF33E0F4CF70D0E0EF
:1018F000809177038295807F0E944B0CDE01AA0FB6
:10190000BB1FA35FBE4F11969C938E93219680912F
:101910007D030E944B0CFE01EE0FFF1FE35FFE4FA5
:1019200091838083DF91CF91089580917803909186
:1019300079039F770E94FE02809377038F3029F40A
:1019400080917D038695805804C099E0899F802D01
:10195000112480937C03F8940E945C0C789480910D
:10196000ED038132E1F480917C039FEF980F9E3F5D
:1019700078F08091B0008F7D8093B00061E080911D
:101980007C03811101C060E083E00E945A1C08952D
:101990008093B4008091B00080628093B00008957D
:1019A000FF920F931F93CF93DF930BEE13E0C0E0F2
:1019B000D0E0B3E0FB2E8C2FD801ED918D019E2F4E
:1019C000907F9031F1F4EF70F0E0EE0FFF1FE35FD6
:1019D000FE4F208131816F2D0E943B20E92FF0E0E6
:1019E000EE0FFF1FEC56FD4F61E080819181821761
:1019F000930708F060E0FE01EE55FD4F80810E94E4
:101A00005A1C2196C830D105B1F6CDB7DEB7E5E056
:101A10000C94C5200F931F93CF93DF9303E513E03E
:101A2000C0E0D0E02091F903822F8F7090E0C817BA
:101A3000D907E9F00196C817D90711F42033B8F493
:101A4000F801808191819F70892B79F0F894F801D9
:101A5000808191819F700E94B202FE01EE0FFF1FF4
:101A6000E35FFE4F9183808378940E94D00C21968F
:101A70000E5F1F4FC031D105A9F6DF91CF911F91A5
:101A80000F910895FF920F931F93CF93DF9381ECF3
:101A900093E00E94AA01809306019091F903292FF7
:101AA0002F70281304C081E0820F809306019053A9
:101AB0009F3060F44091060130E0842F90E0019760
:101AC0002817390719F44F5F4093060180910601EA
:101AD000813118F080E180930601ECE1F3E0DF0151
:101AE00012971C92DF0111971C921082339683E0AB
:101AF000E433F807A1F74FEF3FEFACEAB2E00BEEAB
:101B000013E02FEFE80189918E018031F8F490E025
:101B1000FD0132976081FC01EE0FFF1FE80FF91FF6
:101B2000E65EFC4F8081862B8083CD010197EC011E
:101B300058818181852B81839C918281892B82832D
:101B40006095509590952923352346231396D3E02D
:101B5000033F1D07B9F640931703309318032093F2
:101B60001903C2EAD2E00BEE13E0F12CF8018191E7
:101B70008F01823230F08632B8F0863211F460E0A4
:101B800010C0F6E0FF1204C08091C1008F7E06C035
:101B900087E0F81205C08091C100877F8093C10063
:101BA00061E088810E94211CF3942196E8E0FE12F6
:101BB000DDCF8091EB03803231F461E089E00E9457
:101BC0005A1C82E801C082E08093800081E080930B
:101BD0007503809374038091ED03813211F0873295
:101BE000D9F461E083E00E94211C60E083E00E9460
:101BF0005A1C8091ED03813231F481E08093B00072
:101C00008093B10009C082E08093B00085E08093AA
:101C1000B1008EE38093B3008AE1809381008FEF5F
:101C20009FEF909389008093880080ED97E09093D8
:101C300087008093860080E49CE99093080180935C
:101C400007019093160380931503109276038091F9
:101C50006F00816080936F008091F80383FF0DC057
:101C600080915303909154039F70892B31F00E940F
:101C70000A0D1092740310927503CDB7DEB7E5E03C
:101C80000C94C520CF93C82F8091F0038B3221F4A0
:101C90006C2F8FE00E945A1C8091ED03873249F42B
:101CA0008091B000CC2311F0806101C08F7E8093C1
:101CB000B000CF910895A4E2B0E0E1E6FEE00C941C
:101CC0009C206B017C010E945D1B4B015C0181E04B
:101CD0000E94640483E08093BE030E9462056AEC64
:101CE00071E082E194E00E942B1D7BE1272EE0E56C
:101CF0003E2EF7E47F2EA6E44A2EB5E55B2EC114F6
:101D0000D104E104F10469F00E945D1B68197909AE
:101D10008A099B096C157D058E059F0510F080E0F2
:101D2000D5C08091BE03843051F768ED71E082E147
:101D300094E00E942B1D8FE70E944B030E945E03DC
:101D40008CA3823601F501EC13E00E945E03D801FA
:101D50008D938D01B3E00A3E1B07B9F78091C10353
:101D6000883309F0ADC061EE71E082E194E00E9439
:101D70002B1D82E48CA361E0CE0184960E94C105F4
:101D80005D9A81E0A3C0803741F0893611F581E08A
:101D90000E946B0889E4898304C03982C12CD12C4C
:101DA00076019091BD038091F803992311F080682A
:101DB00001C08F778093F803EAEEF3E0DE0112961C
:101DC000822D01900D928A95E1F76CE1CE0101968A
:101DD00075C08437E1F4E4E5E98383E08A8380E831
:101DE0008B8388E08C838FE08D838EE1EDE2F1E0E0
:101DF000DE01169601900D928A95E1F763E2CE011D
:101E000001960E94C105C12CD12C760159C085379D
:101E100089F40AEE13E00E945E03D8018D938D01D0
:101E2000B4E005301B07B9F761E080E00E94BD0710
:101E30005CA241C08636B9F44982E3E5F3E0AE0125
:101E40004D5F5F4F208131813296CA010197DC01DD
:101E50003C93DA012C934E5F5F4FB3E0E337FB070F
:101E600089F761E2B3CF8736C9F403E513E00E9436
:101E70005E03682E0E945E03262D30E0322F22275B
:101E8000280F311DF801219331938F01F3E00337BF
:101E90001F0769F77CA20E9457080DC0873481F4A0
:101EA000E3E5F3E01192119283E0E337F807D1F70D
:101EB0000E9457087CA261E0CE0184960E94C10571
:101EC00083E08093BE030E943F0519CFA496E2E110
:101ED0000C94B8201F93CF93DF93C82FD62F61E0C7
:101EE0000E94211C61E08C2F0E945A1C61E08D2F02
:101EF0000E945A1C8AE090E00E94B21B8D2F0E9423
:101F00008D1C892B71F060E08C2F0E945A1C8AE096
:101F100090E00E94B21B8D2F0E948D1C11E0892B36
:101F200009F010E060E08C2F0E94211C60E08C2FF3
:101F30000E945A1C60E08D2F0E945A1C812FDF9155
:101F4000CF911F91089580E48093BA001092BD0054
:101F50008DE990E09093B6038093B50310925003FF
:101F600015E004E0C2E0FC2E80915003813039F48A
:101F700080E00E946404F09250035E98F5CFC09117
:101F80005003C33061F45D98809192030E948603F0
:101F9000C093BE030E943F0500935003E5CF80919C
:101FA0005003843009F78091BE038430E9F68FE74F
:101FB0000E944B03C0E0D3E0E091E903E770F0E05A
:101FC000E656FD4F808190E09E0120503340281757
:101FD000390724F40E945E038993EECF10935003D7
:101FE0005D9AC2CFAAE2B0E0E8EFFFE00C94AB202C
:101FF0001FEF198389E2E1ECF3E0DE011296019014
:102000000D928A95E1F721E04AE2BE016F5F7F4FB2
:1020100080E20E94480A81110EC021E041E0BE0129
:102020006F5F7F4F80E20E949D0A811104C082E0B1
:102030008093500302C0109350038091500382306C
:1020400051F00E945D1B60934C0370934D0380938D
:102050004E0390934F03AA96E3E00C94C720A1E0AF
:10206000B0E0E5E3F0E10C94AC20809150038230C5
:10207000D9F480919203805A898321E041E0BE0126
:102080006F5F7F4F80E20E94480A882369F08FEFDC
:10209000809350030E945D1B60934C0370934D032B
:1020A00080934E0390934F032196E2E00C94C82056
:1020B000A1E0B0E0EEE5F0E10C94AC20809150039B
:1020C0008230D1F421E041E0BE016F5F7F4F80E2BA
:1020D0000E949D0A882371F08FEF809350030E9425
:1020E0005D1B60934C0370934D0380934E0390935C
:1020F0004F0302C0898101C08FEF2196E2E00C946A
:10210000C820A2E2B0E0E7E8F0E10C949C209E0138
:102110002F5F3F4F80E1D9011D928A95E9F76CEE60
:1021200071E082E194E029A33AA30E942B1D0E9452
:1021300062051D8A1E8A1F8A188E312C212C00E010
:10214000812C912C5401412C84E7582E8BE8682E69
:1021500082E3782E90E5C92E93ECD92EE12CF12C58
:1021600084EF91E0A0E0B0E08D8F9E8FAF8FB8A399
:1021700080E09EECADEEB4E3898F9A8FAB8FBC8F7D
:1021800080E094E7ABE8B2E3898B9A8BAB8BBC8B96
:1021900082E194E00E94F71D892B09F4E1C082E1FD
:1021A00094E00E94241E9C0133272C32310509F44F
:1021B00042C0ACF42332310509F0ABC019821A8257
:1021C0001B821C821D821E821F82188619861A8617
:1021D0001B861C861D861E861F86188A60C02434B6
:1021E000310529F02335310509F4B2C092C064E409
:1021F00082E194E00E940F1D2AE030E040E054E7C5
:102200006BE872E382E194E00E948B1D6CE282E154
:1022100094E00E940F1D2AE030E040E05EEC6DEE9D
:1022200074E382E194E00E948B1D6CE282E194E011
:102230000E943D1DADCF0F5F043009F0A9CF298169
:102240003A814B815C81A8EEB3E00E941820698B33
:102250007A8B8B8B9C8B2D813E814F8158850E9480
:102260001820698F7A8F8B8F9C8F29853A854B85B3
:102270005C852D8F3E8F4F8F58A32D853E854F85D2
:1022800058890E9418206B017C0160323EE473077C
:102290008105910530F462E38CE10E94730300E054
:1022A00077CF603345E774078105910510F462E24A
:1022B000F3CF60345CE975078105910510F466E29F
:1022C000EBCF80E5C81683ECD806E104F10410F4E6
:1022D00062E1E2CF90E6C9169AEED906E104F10474
:1022E00010F465E1D9CFA0E7CA16A1E1DA06A1E0B2
:1022F000EA06F10410F461E0CFCFB0EACB16B6E8FD
:10230000DB06B1E0EB06F10410F463E0C5CF65E055
:10231000C3CF10ED180F1A3008F03ACFE1E0F0E02B
:10232000EC0FFD1F24E0029FE00DF11D1124208120
:10233000318142815381AAE0B0E00E941820610FF0
:10234000711D811D911D608371838283938320CFD2
:1023500049885A886B887C88812C912C540118CF2D
:1023600081149104A104B10489F4C301B2010E9453
:10237000F90361E070E080E090E00E948C1B1D8A10
:102380001E8A1F8A188E312C22242A948D8D9E8DB0
:10239000AF8DB8A188169906AA06BB06D0F40E9494
:1023A0009C032D893E894F89588D280F311D411D71
:1023B000511D2D8B3E8B4F8B588F381608F4382EBD
:1023C000821508F4282E3FEF831A930AA30AB30A52
:1023D00056C0C301B20128EE33E040E050E00E9455
:1023E0005B20BA01A9012AE030E082E194E00E947A
:1023F000D91D6CE282E194E00E940F1D4AE050E09A
:10240000632D82E194E00E94E81D6CE282E194E099
:102410000E940F1D6D897E898F89988DA501940179
:102420000E945B20BA01A9012AE030E082E194E039
:102430000E94D91D6CE282E194E00E940F1D4AE0E7
:1024400050E0622D82E194E00E94E81D6CE282E19E
:1024500094E00E943D1D4C0C5D1C6E1C7F1C898D00
:102460009A8DAB8DBC8D84159505A605B70520F416
:1024700049885A886B887C88812C912C5401298941
:102480003A894B895C89283E33404105510509F062
:102490007FCEA296E2E10C94B820A1E0B0E0E3E5A3
:1024A000F2E10C94AC2080E00E94900161E085E0B4
:1024B0000E94211C61E086E00E94211C0E946701AD
:1024C00060E080E00E94211C61E081E00E94211C0C
:1024D00040E052EC61E070E082E194E00E943F1F36
:1024E0000E94A9080E945C0869EF71E082E194E013
:1024F0000E940C1D80E893E00E94660760E172E094
:1025000082E194E00E940C1D4AE050E067E070E038
:1025100082E194E00E94C11D0E947C0178945E9A41
:1025200063E183E00E946A0F882329F05E985D983A
:102530000E948110FBCF62E189E00E946A0F811145
:1025400004C00E944508811119C063E572E082E170
:1025500094E00E940C1D60E070E0CB010E945B0ED5
:10256000882349F00E94520868E172E082E194E019
:102570000E942B1D5D9A0E94420D10C00E94420DC8
:102580008091EC03823209F0CAC08091EE0383325D
:1025900009F0C5C08091F80381FDC7C08091EC03AC
:1025A000823231F58091EE03833211F581E00E9491
:1025B000B3088091F80382FF08C063E372E082E110
:1025C00094E00E942B1D0E94A30F64E170E080E064
:1025D00090E00E948C1B21E041E0BE016F5F7F4FC5
:1025E00080E20E949D0A811103C081E08093500324
:1025F0006EE372E082E194E00E940C1D8FE00E9485
:10260000900180E00E9464041092920380E00E9496
:10261000860380E0883170F08093D40283E0809359
:10262000BE030E94620580915003882371F00E94CE
:10263000F20F0BC021E0280FE82FF0E0EF53FC4F22
:102640009785992349F3822FE5CF8091F203982F44
:102650009D7F983229F440E052EC61E070E027C0A1
:10266000893271F440EA56E861E070E082E194E07A
:102670000E943F1F8091C20080628093C2001BC0F5
:102680008091E9038871803129F440E855E260E0E7
:1026900070E00DC04091C2035091C3036091C40328
:1026A0007091C5034A3051056105710570F382E1EF
:1026B00094E00E943F1F82E194E00E94F71D892B65
:1026C00029F082E194E00E94241EF5CF8091F1036D
:1026D000843229F08091C1008F7E8093C100809167
:1026E000F203853241F08852833028F08091C10096
:1026F000877F8093C1001092D6021092D50210926B
:1027000052030E94691B60938E0370938F03809322
:102710009003909391032196E2E00C94C82080915D
:10272000F8038B7F8093F80335CF82FD37CF64EFBA
:1027300071E080E090E00E945B0E882309F42ECFC8
:102740000E94520868E172E082E194E00E942B1D31
:102750000E94420D5D9A22CFCF93DF9382E194E0F5
:102760000E94F71D892BE9F0C091D502D0E0CE017F
:1027700001968F7199272091D60230E08217930736
:1027800081F082E194E00E94241EC952DD4F8883CB
:102790008091D50290E001968F7199278093D502A0
:1027A000DDCFDF91CF910895A0E0B0E0EAEDF3E155
:1027B0000C94A620D82FC62F0E94691B0091AB0352
:1027C0001091AC032091AD033091AE036B017C01FD
:1027D000C01AD10AE20AF30A9701860141E1C41640
:1027E00047E2D406E104F10408F4D1C16093AB03DD
:1027F0007093AC038093AD039093AE0380910D0171
:1028000090910E01880F991F80939303892F8770F1
:1028100020919403287F282B2093940380910F010B
:1028200090911001880F991F382F330F330F330FFA
:102830002770232B20939403282F22952695277009
:1028400080919503807C9770990F990F990F822B37
:10285000892B809395032091110130911201220F51
:10286000331F922F9295990F990F907C8F73892B1C
:1028700080939503932F9295990F990F907C822FB7
:1028800086958695892B8093960332FB882780F95D
:10289000209197032E7F282B20939703809113017B
:1028A00090911401880F991F382F330F2170232B1B
:1028B00020939703382F331F3327331F209198031A
:1028C000207F892F8770880F232B282B2093980334
:1028D0008091150190911601880F991F382F32951C
:1028E000307F2F70232B20939803382F32953F7021
:1028F000209199032078892F87708295807F232BE0
:10290000282B209399038091170190911801880F2B
:10291000991F2F7720939903292F279522272795F1
:102920008695822B80939A03892F869583702091B8
:102930009B032C7F282B20939B038091190190915E
:102940001A01880F991F382F330F330F2370232B51
:1029500020939B03382F329536953695337020910E
:102960009C03207E892F8770880F880F232B282BAC
:1029700020939C0380911B0190911C01880F991F4B
:10298000382F3295330F307E2F71232B20939C03E9
:102990009295990F907E869586958695892B809342
:1029A0009D0380911D0190911E01880F991F8093B6
:1029B0009E03892F877020919F03287F282B2093C7
:1029C0009F0380911F0190912001880F991F382F3C
:1029D000330F330F330F2770232B20939F03282FA0
:1029E0002295269527708091A003807C9770990F7F
:1029F000990F990F822B892B8093A003209121019D
:102A000030912201220F331F922F9295990F990F27
:102A1000907C8F73892B8093A003932F9295990FAD
:102A2000990F907C822F86958695892B8093A103A0
:102A300032FB882780F92091A2032E7F282B209338
:102A4000A2038091230190912401880F991F382FB0
:102A5000330F2170232B2093A203382F331F3327EA
:102A6000331F2091A303207F892F8770880F232B8A
:102A7000282B2093A3038091250190912601880F94
:102A8000991F382F3295307F2F70232B2093A3036B
:102A9000382F32953F702091A4032078892F8770BA
:102AA0008295807F232B282B2093A40380912701DC
:102AB00090912801880F991F2F772093A403292F25
:102AC0002795222727958695822B8093A503969597
:102AD00093708091A6038C7F892B8093A60320910D
:102AE000290130912A01220F331F922F990F990F3C
:102AF0008370892B8093A6032295269526952370B3
:102B00008091A703807E932F9770990F990F822B46
:102B1000892B8093A70320912B0130912C01220F48
:102B2000331F922F9295990F907E8F71892B8093EE
:102B3000A703832F8295880F807E2695269526955C
:102B4000282B2093A803DD2311F088E001C080E04A
:102B5000CC2311F094E001C090E0892B8093A9036D
:102B60006FE070E082E194E00E940201C3E9D3E0EB
:102B7000699182E194E00E94511E83E0CA3AD8072D
:102B8000B9F760E070E082E194E00E940201CDB705
:102B9000DEB7E8E00C94C220CF93C82F682F82E103
:102BA00094E00E94511E8C2F0E940A01CF9108953B
:102BB000A0E0B0E0EEEDF5E10C94A620C82F0E9455
:102BC000691B0091AB031091AC032091AD033091D0
:102BD000AE036B017C01C01AD10AE20AF30A970125
:102BE000860141E1C41647E2D406E104F10408F489
:102BF00045C06093AB037093AC038093AD03909397
:102C0000AE031092C0031092BF0388EA0E94CC1555
:102C1000CC2311F081E801C081E00E94CC1580E155
:102C20000E94CC1500E010E0F801EE0FFF1FE35FFB
:102C3000FE4F808191810E94DD02EC01B3E0CC0F58
:102C4000DD1FBA95E1F78D2F0E94CC158C2F0E94C5
:102C5000CC150F5F1F4F0031110531F76091C00394
:102C600070E082E194E00E94FA006091BF037091ED
:102C7000C003772782E194E00E94FA00CDB7DEB767
:102C8000E8E00C94C220AAE1B0E0E9E4F6E10C949B
:102C90009E200E949B008CE00E946D0381110BC05E
:102CA0006CE872E082E194E00E942B1D80E00E94BB
:102CB00064040E9462050E94AC130E94691B0E947A
:102CC000581091E0853009F090E01FEF8091BE032D
:102CD000843009F4FEC19111FCC17CC00E94A003A4
:102CE00090937B0380937A035D9AC0928E03D09277
:102CF0008F03E0929003F092910310925103809120
:102D0000780390917903880F991F816090937903DC
:102D1000809378035E9880E00E94420E80910003C9
:102D2000982F9E7309F02CC2F8948091E90341E03A
:102D300053E06DE071E087700E942C020E945C0CF1
:102D400078949091000380914A0390FF13C28111FF
:102D500024C093E5E92E93E0F92E00E010E0F7019E
:102D60008081918194FD0CC0F801EE0FFF1FE35F9D
:102D7000FE4F808191810E94DD02D7018D939C934B
:102D80000F5F1F4FB2E0EB0EF11C0031110539F758
:102D90000E94570881E080934A0380915203811179
:102DA00003C081E080935203109273031092750365
:102DB000109274038091E903887109F009C20E949E
:102DC000D00C83E08093BE030E943F0581E0809396
:102DD0004B035D980E94691B4B015C010E945D1BC7
:102DE0006B017C0180915103823008F063C04090F8
:102DF0008E0350908F0360909003709091038091A8
:102E00008A0390918B03A0918C03B0918D0384155C
:102E10009505A605B70509F44DC081EC93E00E9425
:102E2000BA016C5D7540810991099501840104190D
:102E30001509260937096017710782079307D0F52E
:102E400040928A0350928B0360928C0370928D03A0
:102E50000E949C03282F80937E0380917F03909192
:102E60008003820F911D9093800380937F03609174
:102E700081036F5F609381036930E0F070E00E942E
:102E800047207093800360937F0380917D03E3E08C
:102E90008E9F600D711D11247695679576956795C7
:102EA00060937D030E94950C1092800310927F0323
:102EB00010928103809152030091D402882351F132
:102EC00010915103101708F035C240908E035090B6
:102ED0008F036090900370909103A50194012419D1
:102EE0003509460957092F8B388F498F5A8F81EC46
:102EF00093E00E94BA0168517C4F8F4F9F4F2F89FA
:102F0000388D498D5A8D621773078407950708F429
:102F1000D8C110C280918E0390918F03A09190032D
:102F2000B091910375016401C81AD90AEA0AFB0A33
:102F300081EC93E00E94BA019B01AC01A02FB0E0AC
:102F40000E9418206C157D058E059F0558F480920F
:102F50008E0390928F03A0929003B092910381E030
:102F600080934B0380917403811116C08091F2030A
:102F7000883219F40E94F40A0FC0893239F4609142
:102F80005103809173030E94D41306C08A3221F446
:102F9000809173030E94D81580914B03882309F414
:102FA00072C0E0919203EF5FE0939203E83131F059
:102FB000F0E0EF53FC4F8785811102C0109292031D
:102FC0008091FA039091FB03A091FC03B091FD0363
:102FD000892B8A2B8B2B09F44EC080918203909110
:102FE0008303A0918403B0918503892B8A2B8B2BBB
:102FF00009F441C00E945206082F10E020910901F7
:1030000030910A0136952795369527952C5E3F4FCE
:103010002017310770F40E945D1B68517C4F8F4F61
:103020009F4F6093820370938303809384039093F4
:103030008503C801880F991F880F991F40910901C6
:1030400050910A019A01220F331F240F351F820F5E
:10305000931F969587959695879590930A018093EF
:1030600009016091C6037091C7038091C8039091D4
:10307000C9030E94F903809192030E9486030E9473
:103080002F1010924B03809150038F3F09F04DC2D7
:103090000E945D1B00914C0310914D0320914E0343
:1030A00030914F03601B710B820B930B693E734091
:1030B0008105910508F439C20E945D1B60934C03A1
:1030C00070934D0380934E0390934F030E94F20F31
:1030D0002CC20E94691B6B017C018091BE0384306D
:1030E000D1F48FE70E944B0300E013E0E091E90385
:1030F000E770F0E0E656FD4F808190E098012050A7
:103100003340281739070CF0E9CD0E945E03D8013F
:103110008D938D01EBCFE091E903E770F0E0E65687
:10312000FD4F40814F5F21E0BE016F5F7F4F80E226
:103130000E949D0A882371F0109350030E945D1B2A
:1031400060934C0370934D0380934E0390934F0311
:1031500090E0BCCDE091E903E770F0E0E656FD4F6A
:10316000408150E0BE016E5F7F4F80E093E00E949F
:10317000D920BBCD882309F410CE10924A030DCE7E
:10318000982F9873983309F008CE9091F702892709
:1031900087FF03CE90589093F7028091F203853217
:1031A00009F0FBCD10E0212F30E080910003877003
:1031B00090E0821793070CF4F0CD1F5FE12FF0E051
:1031C000E050FD4F608182E194E00E94511EEBCF00
:1031D0008091F70290910003982796FD66C0807C4D
:1031E00090E489278093F7028091D6023091D5022E
:1031F0008317D1F0E8EFF2E020E02F5F90E0DC01F0
:10320000A952BD4F4C91419301968F719927283057
:1032100011F08313F2CF8093D602295C8091F702DC
:10322000282B2093F70241C080917E038093F802FF
:103230008091EC03863211F482E105C08091EF03A6
:10324000863251F48EE00E94B61C9595879595952F
:1032500087958093F90202C01092F9028091EE03E3
:10326000863211F483E105C08091F003863251F477
:103270008FE00E94B61C95958795959587958093CC
:10328000FA0202C01092FA0280917A0390917B03B5
:103290009093FB028093FC028091780390917903D4
:1032A0009F770E94FE028093FD0269E087EF92E023
:1032B0000E947A050E94E905811181CD0E94AC131C
:1032C000F9CF8091780390917903880F991F90939B
:1032D00079038093780381E080934B03111110C030
:1032E000C0928603D0928703E0928803F09289030C
:1032F000109282031092830310928403109285032C
:103300001F5F1093510381EC93E00E94BA01640D9A
:10331000751D861D971D60938E0370938F03809398
:103320009003909391035E9A81E00E94420E0E9466
:10333000950C03C0101709F4A7C08091510388238E
:1033400009F410CE809102048823D9F09091730380
:10335000911117C0409186035091870360918803B3
:103360007091890346015701841A950AA60AB70A83
:1033700090E00E942301681579058A059B0508F4F1
:10338000B5C0809104048823D9F090917503911100
:1033900017C0409186035091870360918803709114
:1033A000890346015701841A950AA60AB70A90E0D4
:1033B0000E942301681579058A059B0508F4ADC0B4
:1033C000809103048823D9F090917403911117C060
:1033D000409186035091870360918803709189031F
:1033E00046015701841A950AA60AB70A90E00E947E
:1033F0002301681579058A059B0508F492C0809120
:10340000FA039091FB03A091FC03B091FD03892B7B
:103410008A2B8B2B09F4A6CD809182039091830394
:10342000A0918403B09185030097A105B10509F42B
:1034300099CDC81AD90AEA0AFB0AF7FC93CD809104
:10344000F803829581700E94950680E00E946404D2
:103450000E943F050E945D1B6B017C012091FF03D0
:1034600030E0A8EEB3E00E940920C60ED71EE81E89
:10347000F91E6894C0F8C0928203D0928303E09250
:103480008403F09285036ECD80918E0390918F031B
:10349000A0919003B091910324013501481A590A73
:1034A0006A0A7B0A81EC93E00E94BA019B01AC019D
:1034B000A12FB0E00E9418206415750586059705B8
:1034C00008F03BCF109279031092780381E080934B
:1034D0004B0310927D030E94950C80928E03909274
:1034E0008F03A0929003B092910327CF81E0809345
:1034F00073030E940A0D8091FE030E9448016C0D27
:103500007D1D8E1D9F1D61606093820370938303F8
:10351000809384039093850334CF81E08093750377
:103520004FCF81E0809374036ACF6A96E0E10C94F8
:10353000BA208230E8F4E82FF0E0EE0FFF1FEB5FD7
:10354000FB4F71836083813041F0809169008C7FF3
:10355000842B80936900E89A089580916900440F54
:10356000551F440F551F837F842B80936900E99A70
:1035700008951F920F920FB60F9211242F933F932D
:103580004F935F936F937F938F939F93AF93BF936B
:10359000EF93FF938091050490910604892B29F005
:1035A000E0910504F09106040995FF91EF91BF9118
:1035B000AF919F918F917F916F915F914F913F91CB
:1035C0002F910F900FBE0F901F9018951F920F9282
:1035D0000FB60F9211242F933F934F935F936F93E6
:1035E0007F938F939F93AF93BF93EF93FF938091BC
:1035F000070490910804892B29F0E0910704F091C9
:1036000008040995FF91EF91BF91AF919F918F9120
:103610007F916F915F914F913F912F910F900FBECE
:103620000F901F9018951F920F920FB60F921124B2
:103630002F933F938F939F93AF93BF9380910A04EF
:1036400090910B04A0910C04B0910D0430910904E9
:1036500023E0230F2D3720F40196A11DB11D05C0D5
:1036600026E8230F0296A11DB11D20930904809323
:103670000A0490930B04A0930C04B0930D04809162
:103680000E0490910F04A0911004B09111040196C2
:10369000A11DB11D80930E0490930F04A0931004FC
:1036A000B0931104BF91AF919F918F913F912F9152
:1036B0000F900FBE0F901F9018952FB7F894609140
:1036C0000A0470910B0480910C0490910D042FBF9B
:1036D00008953FB7F89480910E0490910F04A09143
:1036E0001004B091110426B5A89B05C02F3F19F016
:1036F0000196A11DB11D3FBF6627782F892F9A2FF4
:10370000620F711D811D911D42E0660F771F881F9A
:10371000991F4A95D1F70895CF92DF92EF92FF92C9
:10372000CF93DF936B017C010E94691BEB01C114F5
:10373000D104E104F10479F00E94691B6C1B7D0B3C
:10374000683E7340A0F381E0C81AD108E108F1088F
:10375000C851DC4FECCFDF91CF91FF90EF90DF901D
:10376000CF9008950197009739F0880F991F880F1F
:10377000991F02970197F1F70895789484B58260B4
:1037800084BD84B5816084BD85B5826085BD85B505
:10379000816085BDEEE6F0E0808181608083E1E8B4
:1037A000F0E01082808182608083808181608083EC
:1037B000E0E8F0E0808181608083E1EBF0E08081EF
:1037C00084608083E0EBF0E0808181608083EAE7C1
:1037D000F0E080818460808380818260808380814A
:1037E000816080838081806880831092C100089509
:1037F000833081F028F4813099F08230A1F008956F
:103800008630A9F08730B9F08430D1F480918000FF
:103810008F7D03C0809180008F7780938000089512
:1038200084B58F7702C084B58F7D84BD0895809163
:10383000B0008F7703C08091B0008F7D8093B0007F
:103840000895CF93DF9390E0FC01E458FF4F24915B
:10385000FC01E057FF4F8491882349F190E0880FE5
:10386000991FFC01E854FF4FA591B49182559F4FD9
:10387000FC01C591D4919FB7611108C0F8948C9157
:10388000209582238C93888182230AC0623051F470
:10389000F8948C91322F309583238C938881822BDE
:1038A000888304C0F8948C91822B8C939FBFDF9106
:1038B000CF910895A1E0B0E0E0E6FCE10C94AA20ED
:1038C000282F30E0F901E859FF4F8491F901E458BD
:1038D000FF4F1491F901E057FF4F04910023C9F005
:1038E000882321F069830E94F81B6981E02FF0E0B2
:1038F000EE0FFF1FE255FF4FA591B4919FB7F894CB
:103900008C91611103C01095812301C0812B8C9390
:103910009FBF2196E4E00C94C620CF93DF93282F1D
:1039200030E0F901E859FF4F8491F901E458FF4F65
:10393000D491F901E057FF4FC491CC2391F081114C
:103940000E94F81BEC2FF0E0EE0FFF1FEC55FF4F2D
:10395000A591B4912C912D2381E090E021F480E099
:1039600002C080E090E0DF91CF9108958E3008F0A2
:103970008E5087702091BD0190E4299F9001112401
:10398000822B80937C0080917A00806480937A00FF
:1039900080917A0086FDFCCF80917800209179009B
:1039A00090E0922B0895A0E0B0E0E9EDFCE10C94EA
:1039B000A6206C017A01EB01E60EF71E00E010E094
:1039C000CE15DF0561F06991D601ED91FC91019072
:1039D000F081E02DC6010995080F191FF1CFC8012C
:1039E000CDB7DEB7E8E00C94C2206115710589F00F
:1039F000DB010D900020E9F7AD0141505109461B54
:103A0000570BDC01ED91FC910280F381E02D0995CB
:103A1000089580E090E008950E94F51C0895DC016F
:103A2000ED91FC910190F081E02D099508950F939F
:103A30001F93CF93DF93EC016DE00E940F1D8C016B
:103A40006AE0CE010E940F1D800F911FDF91CF9180
:103A50001F910F9108950F931F93CF93DF93EC0164
:103A60000E94F51C8C01CE010E94171D800F911F32
:103A7000DF91CF911F910F9108950F931F93CF93D3
:103A8000DF93EC010E940F1D8C01CE010E94171DD7
:103A9000800F911FDF91CF911F910F910895A1E2A7
:103AA000B0E0E5E5FDE10C94A2207C01C42EE52FF9
:103AB000CB01D22E19A221E02D1510F02AE0D22E32
:103AC0008E010F5D1F4F8D2C912CA12CB12C6C2DD4
:103AD0007E2FA50194010E945B208C2DD29E80191F
:103AE0001124015011098A3010F4805D01C0895CF5
:103AF000F8018083211531054105510521F0C22EC1
:103B0000E32FCA01E4CFB801C7010E94F51CA196BA
:103B1000ECE00C94BE20A0E0B0E0E1E9FDE10C9403
:103B2000A620EC016A017B012115310541F4E881F1
:103B3000F9810190F081E02D642F09951DC02A3094
:103B40003105A9F477FF12C06DE20E940F1D8C01B0
:103B500044275527BA014C195D096E097F092AE0EF
:103B6000CE010E944F1D800F911F06C02AE0B701B1
:103B7000A601CE010E944F1DCDB7DEB7E8E00C9440
:103B8000C2200F931F93CF93DF93EC019A01AB01F7
:103B9000662757FD6095762F0E948B1D8C01CE0104
:103BA0000E94171D800F911FDF91CF911F910F91E0
:103BB00008952115310549F4DC01ED91FC91019046
:103BC000F081E02D642F099508950E944F1D0895FE
:103BD0009A01462F50E060E070E00E94D91D0895E0
:103BE0009A01AB0160E070E00E94D91D0895FC01CC
:103BF00024853585F901E05CFF4F80819181F901D1
:103C0000EE5BFF4F20813181821B930B8F739927CD
:103C10000895FC0184859585FC01E05CFF4F40819F
:103C20005181FC01EE5BFF4F208131814217530728
:103C300041F00190F081E02DE80FF91F808190E0C4
:103C400008958FEF9FEF0895FC0184859585FC0111
:103C5000E05CFF4F40815181FC01EE5BFF4F208112
:103C600031814217530779F0A081B181A80FB91FA4
:103C70008C91208131812F5F3F4F2F733327318308
:103C8000208390E008958FEF9FEF0895FC0181A1BC
:103C9000882329F0A489B5898C9186FFFBCF11A2D6
:103CA0000895CF93DF93FC0126853785D901A05C69
:103CB000BF4F8D919C91119701968F739927E901C0
:103CC000CE5BDF4F4881598184179507D9F30D905A
:103CD000BC91A02DA20FB31F6C93A685B785A05CE5
:103CE000BF4F11969C938E93A689B7892C9181E042
:103CF00090E0078C02C0880F991F0A94E2F7282BE6
:103D00002C9381E081A30488F589E02D8081806473
:103D1000808381E090E0DF91CF91089508951F9214
:103D20000F920FB60F9211242F933F934F938F93BF
:103D30009F93EF93FF938091C00082FD1CC0409140
:103D4000C6008091B8049091B90401968F739927A9
:103D50002091BA043091BB048217930771F0E0916F
:103D6000B804F091B904E858FB4F40839093B9042C
:103D70008093B80402C08091C600FF91EF919F919B
:103D80008F914F913F912F910F900FBE0F901F90E9
:103D9000189582E194E00E94F71D892B11F00E9492
:103DA0008E1E08951F920F920FB60F9211242F931B
:103DB0003F938F939F93EF93FF93209174043091DF
:103DC000750480917604909177042817390731F4AF
:103DD0008091C1008F7D8093C10014C0E091760472
:103DE000F0917704EC5CFB4F2081809176049091F8
:103DF000770401968F7399279093770480937604C4
:103E00002093C600FF91EF919F918F913F912F9149
:103E10000F900FBE0F901F901895A0E0B0E0E3E167
:103E2000FFE10C94A220FC011382128288EE93E041
:103E3000A0E0B0E084839583A683B78386EC92E00C
:103E4000918380837587648757874687318B208B62
:103E5000138B028BF58AE48AD78AC68AB18EA08E2C
:103E6000938E828E8F85848F8889858F8989868FAE
:103E70008A89878F8B8980A3ECE00C94BE20CF9237
:103E8000DF92EF92FF92CF93DF93EC016A017B0107
:103E9000411581EE580761057105F9F0EC89FD893E
:103EA00081E090E008A002C0880F991F0A94E2F711
:103EB000808360E079E08DE390E0A70196010E94A5
:103EC0005B20215031094109510956954795379595
:103ED0002795211580E1380798F0EC89FD8910823B
:103EE00060E874E88EE190E0A70196010E945B20F3
:103EF0002150310941095109569547953795279524
:103F0000E889F9893083EA89FB89208319A2EE893F
:103F1000FF89408181E090E09C010C8C02C0220F5F
:103F2000331F0A94E2F7422B4083EE89FF894081D8
:103F30009C010D8C02C0220F331F0A94E2F7422B22
:103F40004083EE89FF8940819C010E8C02C0220FC4
:103F5000331F0A94E2F7422B4083EE89FF892081C8
:103F60000F8C02C0880F991F0A94E2F78095822374
:103F70008083DF91CF91FF90EF90DF90CF900895F5
:103F80008F929F92AF92BF92CF92DF92EF92FF9269
:103F90000F931F9381E08F9385E08F9387E08F933A
:103FA00083E08F9384E08F93E6EC8E2E912CF2ECDD
:103FB000AF2EB12CA1ECCA2ED12CB0ECEB2EF12CF3
:103FC00004EC10E025EC30E044E354E068E774E0F2
:103FD00082E194E00E940D1F0F900F900F900F90C0
:103FE0000F901F910F91FF90EF90DF90CF90BF90B7
:103FF000AF909F908F9008950E94BD1B0E944D121C
:10400000C9ECDEE10E9443162097E1F30E94C91E2D
:10401000F9CFA29FB001B39FC001A39F700D811D76
:104020001124911DB29F700D811D1124911D0895C1
:104030000E940920A59F900DB49F900DA49F800D14
:10404000911D11240895B7FF0C9418200E94182088
:10405000821B930B0895DB018F939F930E9418207E
:10406000BF91AF91A29F800D911DA39F900DB29F14
:10407000900D11240895991B79E004C0991F96179B
:1040800008F0961B881F7A95C9F780950895AA1B9A
:10409000BB1B51E107C0AA1FBB1FA617B70710F033
:1040A000A61BB70B881F991F5A95A9F78095909565
:1040B000BC01CD010895A1E21A2EAA1BBB1BFD0174
:1040C0000DC0AA1FBB1FEE1FFF1FA217B307E407F7
:1040D000F50720F0A21BB30BE40BF50B661F771F4F
:1040E000881F991F1A9469F760957095809590952F
:1040F0009B01AC01BD01CF010895052E97FB1EF475
:1041000000940E94942057FD07D00E945B2007FC7A
:1041100003D04EF40C949420509540953095219501
:104120003F4F4F4F5F4F08959095809570956195E3
:104130007F4F8F4F9F4F08952F923F924F925F92E4
:104140006F927F928F929F92AF92BF92CF92DF92A7
:10415000EF92FF920F931F93CF93DF93CDB7DEB70C
:10416000CA1BDB0B0FB6F894DEBF0FBECDBF0994A0
:104170002A88398848885F846E847D848C849B84F7
:10418000AA84B984C884DF80EE80FD800C811B8105
:10419000AA81B981CE0FD11D0FB6F894DEBF0FBE34
:1041A000CDBFED010895EE0FFF1F0590F491E02DB6
:1041B0000994FB01DC0102C001900D924150504076
:1041C000D8F70895F999FECF92BD81BDF89A992745
:1041D00080B50895262FF999FECF1FBA92BD81BDF3
:1041E00020BD0FB6F894FA9AF99A0FBE0196089579
:0441F000F894FFCF71
:1041F4000000BC04200008409CFF0088130002005B
:10420400020002000200020002000200020002009A
:10421400020002000200020002000200020020016B
:10422400220126022102270323032604260526054C
:104234002B0624072507280729072A8025000005BF
:10424400400AA1204EA50020244EA52C2330C012E4
:1042540000001A400AA1204EA5001B1E27522C2341
:10426400308025000005400AA1204EA50020244EE0
:10427400A52C2330004B000006400AD0009D4900C5
:104284007B289D492C233000E1000005400A4501AC
:10429400D7DC03B81E0EBF00232E48E801008A4075
:1042A4000A6001555502AD1E20000023C801545870
:1042B4002074696D656F7574210057616974696E46
:1042C400672062696E640A00476F7420706B740A19
:1042D400006461746120676F6F640A007363616EC8
:1042E4006E6572206D6F6465004F70656E4C52533D
:1042F4006E67205258207374617274696E6720006F
:10430400206F6E20485720005361766564206269EF
:104314006E64206461746120746F20454550524F6F
:104324004D0A004920616D20736C61766500456E0D
:10433400746572696E67206E6F726D616C206D6F4B
:10434400646500454550524F4D2064617461206E90
:104354006F742076616C6964206F722062696E6488
:10436400206A756D70706572207365742C20666F99
:104374007263696E672062696E640A00525820682D
:10438400616E6700B200F4014C0300070B0C1011BE
:104394001500091203130E0F0001020000001000A3
:1043A40000000800200000010000020000000100DD
:1043B400000200000000511ED31CF71D241E091E1C
:0243C400461E93
:107E00000F92CDB7DEB7112484B714BE81FFF1D035
:107E100082E08093C00088E18093C10086E0809377
:107E2000C20080E18093C4008EE0CDD088249924E4
:107E3000CC24C394F5E0DF2EE1E1EE2E73E0F72EC3
:107E4000B6D0082F813479F4B2D08983C2D0898129
:107E5000823811F481E005C0813811F485E001C059
:107E600083E09ED09AC0823411F484E103C085344B
:107E700019F485E0B6D091C0853561F498D0082F0B
:107E800010E095D090E0982E8824802A912A880CC2
:107E9000991C82C0863521F484E0A3D080E0E1CF34
:107EA000843609F04CC083D082D0A82E80D0B82E62
:107EB00000E011E07CD0F80181938F01AE16D1F77C
:107EC00088D0FB2DF53489F4E0E0F1E00BC0F9999E
:107ED000FECF92BC81BC0894811C911C819180BD15
:107EE000FA9AF99AEA1598F358C08B2D863409F05E
:107EF00054C0F401F7BEE89507B600FCFDCFF401CD
:107F0000A0E0B1E02C9130E011968C91119790E0B7
:107F1000982F8827822B932B12960C01C7BEE895C9
:107F20001124329681E0A038B80761F7F401D7BE7A
:107F3000E89507B600FCFDCFE7BEE8952EC0843774
:107F4000F1F435D034D0182F32D0B82E42D0FB2DDA
:107F5000F63421F4F40105914F010CC0FB2DF534EA
:107F600049F4F999FECF92BC81BC0894811C911C04
:107F7000F89A00B5802F14D0115049F70EC08537FC
:107F800039F427D08EE10CD085E90AD08FE069CF93
:107F9000813511F488E017D01CD080E101D050CF9A
:107FA0009091C00095FFFCCF8093C600089580910A
:107FB000C00087FFFCCF8091C00084FD01C0A89560
:107FC0008091C6000895E0E6F0E098E19083808318
:107FD0000895EDDF803219F088E0F5DFFFCF84E10E
:107FE000DFCF1F93182FE3DF1150E9F7F2DF1F9166
:0E7FF0000895282E80E0E7DFEE27FF27099492
:027FFE0001057B
:0400000300007E007B
:00000001FF
